:020000040000FA
:100000000A128A1116281030A6000310A40DA50D9F
:100010000310A00DA10D031C13282308A507220817
:10002000A4070318A50AA60B052808000608A800BF
:1000300083169B0183129F0183169F0107309C004A
:100040008F300F0570388F006528BE003E080319F9
:10005000080001303E02031D3228000000000000AD
:1000600000000800BE0300000000BF01402883120A
:1000700003130330A0000A128A11A00B3D28BF0A07
:100080003F083E02031D37280800BC01BD015C2863
:1000900083120313B430A000DD30A1000A128A11CC
:1000A000A10B4E280A128A11A00B4C280000000058
:1000B0000000BC0A0319BD0A3C083A02A0003D0832
:1000C0003B022004031D482808008F308100A1282E
:1000D0008312B9003908031D702883161B140514F8
:1000E000013083123902031D782883169B1485146E
:1000F000023083123902031D802883161B15051553
:10010000033083123902031D882883169B15851539
:10011000043083123902031D902883161B1605161E
:10012000053083123902031D982883169B16061783
:10013000063083123902031DA02883161B17861769
:1001400008008312AC012C0EA0003030A005CF3087
:1001500083161F058312200483169F00512938102F
:100160003408A0003508A1000A30A200A301032032
:1001700083122408B6002508B7000310370CA1002D
:10018000360CA0000310A10CA00C0310A10CA00CB5
:100190002008A90010302902B810031D0318B81454
:1001A0003C30290238110319D728031C3815B8151B
:1001B000B818381DB811B819381420103818201480
:1001C0000800F8308312B2054030B400B501AF200A
:1001D0008312B2112018B215B21DF328F83032057F
:1001E0000638B2003B292030B400B501AF2083129D
:1001F000B2122018B216B21E0229F83032050238A7
:10020000B2003B291030B400B501AF208312B21305
:100210002018B217B21F1129F83032050538B20084
:100220003B290830B400B501AF208312B310201869
:10023000B314B31C2029F83032050138B2003B2931
:100240000430B400B501AF208312B3112018B315E8
:10025000B31D2F29F83032050438B2003B29023093
:10026000B400B501AF208312B3122018B316B31E29
:100270003B29F830B20503303205A000200CA10064
:10028000A10C210CA100C030A1053F301F052104A5
:100290009F0032194E2983161F13080083161F175B
:1002A00008008312A7019729B000300DA000A00D0F
:1002B000A00D3830A005C7301F0520049F001F1473
:1002C0002A08252083121F151F1964291E08B10052
:1002D0002630290203196E29031C7829831203137F
:1002E0004E30A0000A128A11A00B74290000822946
:1002F000831203131330A0000A128A11A00B7E2967
:10030000000000001F10310808008312AE002E0804
:1003100054218312AF002F08080083169F13080092
:1003200015308312AA0008008D21E1209029942124
:100330000430682083168601043085218312AB00C7
:1003400005302B020319AD29031CAD29A81128087B
:100350008600281728088600B329A81528088600D3
:100360002813280886000230BA00BB0145208312FA
:10037000AD012D08A800280886008B108B130B16E2
:06038000630000009C294F
:02400E007C3FF5
:02401000FF3F70
:00000001FF
